:0400000042EF00F0DB
:10000800F2A402D0166AF2949EAA04D0AECF23F0CE
:06001800010E156E11003F
:10001E00FF0E246EFF0E256EFF0E266EFF0E276E50
:10002E00FF0E1F6EFF0E206E000E216E000E226E52
:10003E00FF0E176EFF0E186E000E196E000E1A6E62
:10004E00FF0E1B6EFF0E1C6E000E1D6E000E1E6E42
:10005E00AC8A900EAB6E948E949C9EAA03D0AECFBB
:06006E0000F0FBD71200B8
:100074000900F5CFE6FF0006FBE10106F9E11200F5
:10008400156A166A720ED36E0F0EC16E070EB46E29
:10009400926A896A936A8A6A800E946E8B6A9D8AD0
:1000A400E00EF26E880ED56ECF0EAF6EAC84B5DF67
:1000B400020E0B6E040E0C6EBA0E0D6E0D2EFED7D4
:1000C4000C2EFCD70B2EFAD700001550010A2CE198
:1000D400156A300E1624F66E010EF76E000EF72226
:1000E400000EF86E000EF8220900F5CF01F0015061
:1000F400231806E1DE0ED76EA80ED66E162A00D09F
:1001040016500E0A11E18A800B0E0B6E260E0C6E31
:100114005D0E0D6E0D2EFED70C2EFCD70B2EFAD7CE
:0C012400000000008A90166AD0D7FFD7B8
:0F013000537A657A616D5F746172756C6A210034
:020000040030CA
:0D000100081F1EFF0381FF0FC00FE00F401E
:00000001FF
